:100000000C9462000C94B31A0C94E01A0C948A00BD
:100010000C948A000C948A000C948A000C948A0038
:100020000C948A000C948A000C948A000C948A0028
:100030000C948A000C948A0B0C948A000C948A000D
:100040000C940D1B0C948A000C94891E0C94CC1EED
:100050000C948A000C948A000C948A000C948A00F8
:100060000C94EB080C948A000000000700020100C9
:100070000003040600000000000000000102040864
:100080001020408001020408102001020408102002
:10009000040404040404040402020202020203032E
:1000A00003030303000000002300260029000000D2
:1000B0000000250028002B0000000000240027007D
:1000C0002A00402011241FBECFEFD8E0DEBFCDBFF5
:1000D00012E0A0E0B1E0E4EFF2E402C005900D927E
:1000E000A43CB107D9F714E0A4ECB2E001C01D9222
:1000F000AE3AB107E1F710E0C4ECD0E004C02297BB
:10010000FE010E945521C23CD107C9F70E947C2004
:100110000C9478210C9400008091B003813019F484
:1001200082E08093B0038091B003833019F484E0BF
:100130008093B0030895A8950895CF93DF93FC01B1
:10014000962F9270862F817060FF20C0992331F026
:100150008091420380831092C40216C0A091C40211
:10016000C091DB03C770D0E0CC56DD4F8881A81763
:1001700010F080E03CC081E08A0F8093C402B0E0C0
:10018000AE50BD4F8C91808381E031C09923C1F086
:1001900090819093C5021092C402292F207E2036B0
:1001A00051F490914203923020F390819F7190938B
:1001B000840393E01AC09E3F39F71092420317C0A0
:1001C0009091C5029F3F01F79091C402993288F641
:1001D00021E0290F2093C4023081E92FF0E0ED5493
:1001E000FC4F3083293281F691E090934203DF91F6
:1001F000CF910895DC01ED91FC910190F081E02D0B
:1002000009950895DC01ED91FC910190F081E02DBC
:10021000099508952091B1033091B203382748E041
:10022000C901880F991F37FF06C09C0151E225279D
:1002300050E1352701C09C01415091F73093B20342
:100240002093B10308958436910520F4BC0180E029
:1002500090E017C09C018E3B910528F42A55310986
:10026000AAE0B0E00CC0823D910528F4245B31097E
:10027000A4E6B0E004C02D5C3109A8E5B2E00E941C
:100280008920A4E6B0E09B01AC010E94982008956B
:1002900090E08C599F4F0E942301089586E080933F
:1002A000DC0380E28093DD0386E28093DE0391E24B
:1002B0009093DF038093E00384E28093E10385E27F
:1002C0008093E203089560E08CE00E941B1C61E0D3
:1002D0008BE00E941B1C61E08DE00E941B1C60E013
:1002E00082E00E941B1C61E084E00E941B1C0895B8
:1002F00042E050E06CE870E080E00E94931A0895BC
:10030000E3E0F0E089E080935700E491E67081E05B
:10031000E63009F080E00895CF93DF93C82F0E9464
:100320008001882381F0DFB781E08093AF03F894E8
:100330000E949B0088E180936000C0936000C1111F
:100340000E949B00DFBFDF91CF910895FC0140A583
:10035000842F877090E0959587950196242F2170C2
:1003600030E0820F931F880F880F08958F929F921D
:10037000AF92BF92CF92DF92EF92FF92CF93FC01A8
:10038000C0A5EC2FE770F0E0EC56FD4FA081B0E087
:10039000C7FF03C024E130E002C02FE030E0FC01E1
:1003A00097A183E1989FF0011124E85AFE4F8080C5
:1003B0009180A280B380A20FB31F20E43FE14DE7FC
:1003C00050E00E94A320A50194010E94DB208C2F05
:1003D000887149F469017A01E0EDCE0EE7E0DE1E96
:1003E000E11CF11C1BC0C7FF05C060E47AE88CE289
:1003F0009EE004C060E07EEE8AEB9BE069017A013A
:10040000F8EBCF0EFBE0DF1EE11CF11CA50194010F
:100410000E94DB20C20ED31EE41EF51EC701B601EA
:1004200069517C4F8F4F9F4F28EE33E040E050E002
:100430000E94DB20A8EEB3E00E949820CF91FF90AD
:10044000EF90DF90CF90BF90AF909F908F900895E6
:10045000DB01FA01582F569590E02481237030E09B
:10046000322F22274081240F311D11963C932E9369
:1004700044814C70218130E060E4469F200D311DA5
:10048000112413963C932E9312974481407322813A
:1004900030E060E1469F200D311D112415963C93FC
:1004A0002E9314974481407C238130E064E0469F82
:1004B000200D311D112417963C932E9316973596D7
:1004C00018969F5F591748F680FF47C040814295B4
:1004D0004695469543702DE431E0429FC001439F0D
:1004E000900D11240C9611969C938E93808190E030
:1004F00074E0969587957A95E1F783709927829FA6
:10050000A001839F500D929F500D1124445F5F4FB7
:1005100013965C934E931297808190E09695879501
:100520009695879583709927829FA001839F500D90
:10053000929F500D1124445F5F4F15965C934E932C
:10054000149740814370429FC001439F900D112436
:100550000C9617969C938E9316970895803223E0FD
:10056000920708F1883E23E0920740F48F519340B0
:10057000E4E096958795EA95E1F70895803D27E0B8
:10058000920718F48C5D93400895883928E092070B
:1005900068F4885C974074E0969587957A95E1F7C2
:1005A0008D509C4F089580E090E008958FEF93E088
:1005B00008958C30910540F4A4E0880F991FAA9506
:1005C000E1F7885D9C4F0895843F23E0920718F47B
:1005D00084529C4F0895811524E0920740F4865779
:1005E000934FF4E0880F991FFA95E1F7089580E999
:1005F00098E008959C013695279525753575821BE1
:10060000930B9C01237333739695879596958795E5
:1006100083739373820F931F9C0154E03695279543
:100620005A95E1F7280F391F2F703F7041E051E0D4
:10063000249FC001259F900D349F900D1124892F78
:1006400008952D98882319F000002B9A02C000000D
:100650002B9800002D9A000008952D9A000083B178
:100660002D980000829581700895CF93DF93D82F45
:100670005C9A2D985C98C8E08D2F80780E942103A9
:10068000DD0FC150C9F72D98DF91CF9108958F7775
:100690000E9435030895CF93DF93D82FC8E08D2FA4
:1006A00080780E942103DD0FC150C9F72D98DF919A
:1006B000CF910895CF93DF932D98C8E080E0D82F95
:1006C000DD0F0E942D038D0FC150C9F7DF91CF912F
:1006D00008950E9447030E945A035C9A0895A1E07E
:1006E000B0E0E5E7F3E00C942C21806869830E9478
:1006F00035036981862F0E944B035C9A2196E2E0C4
:100700000C944821CF93C091BC03C827E82FF0E098
:10071000ED54FC4F678589E70E946F036C2F8DE3D2
:100720000E946F036C2F82E40E946F03CF910895A3
:1007300086E20E9469030895CF938BE20E946903C9
:10074000C82F8CE20E946903282F30E066E03695BE
:1007500027956A95E1F744E0C49FC0011124822BDC
:10076000932BCF910895CF93DF93EC016C818CE1B3
:100770000E946F036D818DE10E946F036E818EE197
:100780000E946F036F8180E20E946F03688581E29F
:100790000E946F03698582E20E946F036A8583E28B
:1007A0000E946F036B8584E20E946F036C8585E273
:1007B0000E946F036D858AE20E946F036E858EE64C
:1007C0000E946F036F858FE60E946F03688980E740
:1007D0000E946F03698981E70E946F036A8982E73B
:1007E0000E946F03DF91CF910895CF92DF92EF9235
:1007F000FF92CF93DF936B017C01C11488E3D8068D
:100800008CE9E8068CE1F80628F5C701B60120E876
:1008100036E948E950E00E94DB20E901689760E88A
:1008200079E687E69FEF0E94AB206C0D7D1D8E1D43
:100830009F1DF2E0660F771F881F991FFA95D1F769
:1008400021E732E040E050E00E94DB20F22EE32E70
:1008500080E421C0C701B60120E03DE241E351E060
:100860000E94DB20E901689760E073ED8EEC9EEF5B
:100870000E94AB206C0D7D1D8E1D9F1D660F771F86
:10088000881F991F21E732E040E050E00E94DB2002
:10089000F22EE32E80E66C2F6F71680F85E70E94C1
:1008A0006F036E2D86E70E946F036F2D87E70E940E
:1008B0006F03DF91CF91FF90EF90DF90CF9008957D
:1008C0008F929F92AF92BF92CF92DF92EF92FF9260
:1008D000CF93DF93D82F83E00E9469038093AE0308
:1008E00084E00E9469038093AD0360E086E00E948B
:1008F0006F0361E087E00E946F036FE789E00E9469
:100900006F0365E08AE00E946F0362E18BE00E9462
:100910006F0365E18CE00E946F036DEF8DE00E9434
:100920006F0360E08EE00E946F03DD2319F085E421
:1009300091E008C02091DA0333E1239FC001112424
:10094000885A9E4F0E94B3036CE880E30E946F03B5
:100950006FE082E30E946F0362E483E30E946F030F
:100960008091DB0387FF02C064E101C06AE084E399
:100970000E946F036AE285E30E946F036DE286E3E3
:100980000E946F0364ED87E30E946F0360E088E3D9
:100990000E946F0360E089E30E946F03D11109C0D8
:1009A000C090BC03D090BD03E090BE03F090BF03A5
:1009B00007C0C5E9CC2EC1ECDC2EED2CCEEDFC2E13
:1009C000CAE38F2C9924AA24BB24682D8C2F0E9463
:1009D0006F03682D85E08C0F0E946F03FE2CED2CB9
:1009E000DC2CCC24CF5FCE3361F76FEF83E40E9421
:1009F0006F036FEF84E40E946F036FEF85E40E9442
:100A00006F036FEF86E40E946F03DD2311F066E051
:100A100002C06091C0038DE60E946F0360E089E729
:100A20000E946F036091C1038AE70E946F0360E038
:100A300083E70E946F0360E084E70E946F03D11197
:100A400009C06091B8037091B9038091BA03909185
:100A5000BB0304C060EC72E98DEE99E10E94F503DE
:100A6000DF91CF91FF90EF90DF90CF90BF90AF904C
:100A70009F908F90089561E087E00E946F0364E289
:100A80008EE70E946F0363E088E00E946F0360E0DE
:100A900088E00E946F0365E087E00E946F0362E0D8
:100AA00085E00E946F0383E00E9469038093AE0398
:100AB00084E00E9469038093AD03089583E00E945F
:100AC00069038093AE0384E00E9469038093AD03C1
:100AD00061E087E00E946F036AE070E080E090E0F0
:100AE0000E94861B0E943B0500000895CF92DF9272
:100AF000FF920F931F93CF93DF931F92CDB7DEB773
:100B0000082F162F8EE399830E946F03F02EC02EBC
:100B10009981D92E8C2D8F19811738F4F6016191A6
:100B20006F018FE70E946F03F5CF64E085E00E94BC
:100B30006F0383E00E9469038093AE0384E00E9408
:100B400069038093AD030E94631B6093A9037093B4
:100B5000AA038093AB039093AC0369E087E00E9403
:100B60006F0381E08093B0030F90DF91CF911F91CD
:100B70000F91FF90DF90CF9008950F931F930E94E5
:100B800076058091B003813099F40E94631B009137
:100B9000A9031091AA032091AB033091AC03601B11
:100BA000710B820B930B603A76488140910548F3B4
:100BB0008091B003813031F468EB71E084E094E01F
:100BC0000E94251D1F910F9108950F931F938091EF
:100BD000B003823021F41092B00381E020C08091F4
:100BE000B0038130D9F40E94631B0091A9031091D6
:100BF000AA032091AB033091AC03601B710B820BF5
:100C0000930B613A76488140910540F061E087E0BE
:100C10000E946F031092B00382E001C080E01F9138
:100C20000F910895EF92FF920F931F93CF93DF934D
:100C30008B019C01442737FD4095542F60E271EAF7
:100C400087E090E00E94FD20E9011C161D0614F0CB
:100C5000C1E0D0E0D80120E231EA47E050E00E9454
:100C6000A3209E01442737FD4095542F0E94FD206C
:100C7000790100E010E00E151F055CF42B9ACE01FF
:100C80000E94AC1B2B98CE010E94AC1B0F5F1F4F24
:100C9000F2CFCDB7DEB7E6E00C944421CF93DF93DB
:100CA000429A6091EC037091ED038091EE03909174
:100CB000EF030E94F50360E089E70E946F0361E0A3
:100CC00070E080E090E00E94861B0E949803C82F8D
:100CD00061E070E080E090E00E94861B0E94980333
:100CE000D0E0C80FD11D61E070E080E090E00E948C
:100CF000861B0E949803C80FD11D61E070E080E060
:100D000090E00E94861B0E94980342989E01280F43
:100D1000311DC9019695879596958795DF91CF915D
:100D20000895CF93C82F429A83E00E94690380936D
:100D3000AE0384E00E9469038093AD0360E086E027
:100D40000E946F0361E087E00E946F036FE789E014
:100D50000E946F0365E08AE00E946F0362E18BE00E
:100D60000E946F0365E18CE00E946F036DEF8DE0E0
:100D70000E946F0360E08EE00E946F036CE280E7E8
:100D80000E946F0360E080E30E946F0360E089E7E8
:100D90000E946F0365E08AE70E946F0362E181E7CA
:100DA0000E946F0362E082E70E946F0360E083E7C6
:100DB0000E946F0360E084E70E946F036091EC0380
:100DC0007091ED038091EE039091EF030E94F50383
:100DD00067E08DE60E946F036AE070E080E090E0DB
:100DE0000E94861B69E087E00E946F036AE070E062
:100DF00080E090E00E94861BCC2369F0C5E1C150E1
:100E000009F459C061E070E088EB91E00E9412069D
:100E10000E949B00F4CF61E070E088E891E00E94BE
:100E200012060E949B0065E08DE60E946F036AE057
:100E300070E080E090E00E94861B61E070E088EB4B
:100E400091E00E9412060E949B0064E08DE60E94E1
:100E50006F036AE070E080E090E00E94861B61E032
:100E600070E08DE591E00E9412060E949B0062E016
:100E70008DE60E946F036AE070E080E090E00E94DF
:100E8000861B61E070E08FEA90E00E9412060E94EB
:100E90009B0060E08DE60E946F036AE070E080E0F6
:100EA00090E00E94861B62E070E085E091E00E9485
:100EB00012060E949B0061E087E00E946F03429847
:100EC000CF910895CF93DF93EC014AE050E06D2F6E
:100ED00070E084E094E00E94EA1D6EE284E094E019
:100EE0000E94091DBE0184E0769567958A95E1F719
:100EF0006F7077274AE050E084E094E00E94EA1D9A
:100F00006EE284E094E00E94091DBE016F707727B5
:100F10004AE050E084E094E00E94EA1DDF91CF9126
:100F20000895D82FC0E0CD1780F4439A64E670E0AE
:100F300080E090E00E94861B439864E670E080E0C9
:100F400090E00E94861BCF5FEECF6CE271E080E004
:100F500090E00E94861BE6CF0F931F93CF93DF9301
:100F6000EC01062F15E0115051F0CE010E946221D4
:100F7000081741F0602FCE010E946A21F4CF82E071
:100F80000E949107DF91CF911F910F910895A0E0EA
:100F9000B0E0EDECF7E00C941E21482E562EC0E098
:100FA000D0E0612C712CE12CF12C00E010E0442009
:100FB00079F081E04816A1F092E0491219C028E4C6
:100FC000622E712C30E2E32EF12C05E413E010C008
:100FD000612C712C6BE1E62EF12C0CED13E008C0B6
:100FE0004DE1642E712C59E2E52EF12C03EB13E058
:100FF00043018C0E9D1E1092B2031092B103340176
:10100000A62CA818B12CC30101966C01AE14BF0424
:10101000A8F4A00EB11E511006C0C3010E946221A7
:10102000F501808305C0F5016081C3010E94AC0712
:10103000F50180810E940A013601E2CFC3015110FF
:1010400018C0C3010E946221B82EC6010E9462210D
:101050002B2D30E0322F2227282B8091B103909145
:10106000B2038217930779F4C0E0D0E0552453947B
:101070009ECF36016091B2030E94AC076091B1032C
:10108000C6010E94AC07D395C13093E0D90708F49C
:101090008ECF852DCDB7DEB7E0E10C943A2160E02C
:1010A00081E00E94C707882331F081E09091B3036B
:1010B000983309F080E0089561E081E00E94C7075D
:1010C000089561E082E00E94C707089560E082E031
:1010D0000E94C707811108C0E5E4F3E01192119264
:1010E00083E0E536F807D1F70895A1E0B0E0EBE73B
:1010F000F8E00C942C2189830E944E0192E0909399
:10110000EA039FEF9093EB039AE09093F40310921D
:10111000F5031092F6031092EC031092ED03109277
:10112000EE031092EF032EE12093F0039093F1036E
:1011300028EB3BE03093F3032093F203898188236B
:1011400071F061E080E00E94C707E5E4F3E01192EE
:10115000119283E0E536F807D1F70E9461082196E5
:10116000E2E00C94482160E080E00E94C707811112
:1011700003C081E00E9475080895CF93C1E08111FA
:1011800001C0C0E06C2F82E10E94541C6C2F83E1EF
:101190000E94541C1092A3031092A2038091B900E4
:1011A0008C6F8093B90080E28093B80085E48093CF
:1011B000BC00CF91089585ED8093BC008091BC0068
:1011C00084FDFCCF0895ECEBF0E0108285E4808391
:1011D0001092A20308951F920F920FB60F9211243E
:1011E0002F933F934F935F936F937F938F939F932F
:1011F000AF93BF93EF93FF93CF93DF931F92CDB73E
:10120000DEB78091B900887F803609F4C7C0A8F5A1
:10121000883209F464C098F4803109F45DC038F470
:10122000882309F4F3C0883009F456C0F1C088312E
:1012300009F455C0803209F0EBC082E0A7C08034C9
:1012400009F477C078F4803309F45FC0883309F07B
:10125000DFC084E08093A1038091A2038B7F809301
:10126000A203D0C0803509F452C0883509F467C0A4
:10127000883409F0CDC085E089C0883909F4C0C040
:10128000A8F4883709F48AC038F4883609F486C08F
:10129000803709F483C0BCC0883809F4B1C08039F4
:1012A00009F47FC0803809F0B3C07BC0803B09F4EB
:1012B00093C038F4803A09F48CC0883A09F48CC0A1
:1012C000A7C0803C09F49EC0883C09F49BC0883BC1
:1012D00009F09EC080E081C08091A60313C0809178
:1012E000A3039FEF980F9093A3038823D1F1E0917C
:1012F000A403F091A503CF0101969093A5038093D9
:10130000A40380818093BB007DC083E03FC0E09157
:10131000A403F091A503CF0101969093A5038093B8
:10132000A4038091BB0080838091A30381508093AC
:10133000A3038091A303823008F064C061C0E091F0
:10134000A403F091A503CF0101969093A503809388
:10135000A4038091BB0080838091A303815080937C
:10136000A3038091A2038B7F8093A2038091A203A9
:1013700080FF4CC08091A2038E7F8093A203809156
:10138000A20382608093A20384EA3DC08093A103FC
:101390008091A2038B7F8093A20338C01092A30395
:1013A00031C0E091A703F091A803309749F18091F3
:1013B000BB0089838091A30391E0980F9093A303CE
:1013C000811102C062E001C060E0CE010196099582
:1013D00015C00E94DB0816C081E0E091A703F091E0
:1013E000A803309769F0882311F063E001C061E041
:1013F000CE010196099599819093BB00811102C09D
:1014000085E801C085EC8093BC0002C00E94DB0827
:101410000F90DF91CF91FF91EF91BF91AF919F918D
:101420008F917F916F915F914F913F912F910F908D
:101430000FBE0F901F9018958F929F92AF92BF9200
:10144000CF92DF92EF92FF92CF93DF93EC010E9455
:10145000631B6B017C014E01A12CB12C8091A20376
:1014600082FF11C02097D1F30E94631B6C197D0984
:101470008E099F0986169706A806B90678F70E9476
:10148000E30881E004C08091A1031092A103DF91E1
:10149000CF91FF90EF90DF90CF90BF90AF909F9053
:1014A0008F900895A2E0B0E0E8E5FAE00C942821DE
:1014B000182F7B01022F047022FD05C080910B01C3
:1014C00090910C0102C080E090E02A8349830E9441
:1014D0001C0A2A814981811136C01092A1034093D0
:1014E000A303F092A503E092A403110F1093A603A7
:1014F0009091A20321FF02C085E001C084E0892B06
:101500008093A2038091A20381FF0BC08091A2036C
:101510008D7F8093A2038091A6038093BB0085EC0E
:1015200001C085EE8093BC00822F817020FF0BC02C
:10153000011105C080910B0190910C0102C080E067
:1015400090E00E941C0A2296E6E00C944421A2E05E
:10155000B0E0EDEAFAE00C942821182F7B01022F6D
:10156000047022FD05C080910B0190910C0102C016
:1015700080E090E02A8349830E941C0A2A814981E5
:10158000811138C01092A1034093A303F092A503E8
:10159000E092A403812F880F81608093A60390912D
:1015A000A20321FF02C085E001C084E0892B809363
:1015B000A2038091A20381FF0BC08091A2038D7FC3
:1015C0008093A2038091A6038093BB0085EC01C0A9
:1015D00085EE8093BC00822F817020FF0BC001112B
:1015E00005C080910B0190910C0102C080E090E059
:1015F0000E941C0A2296E6E00C944421A0E0B0E090
:10160000E4E0FBE00C9426210E94631B00919D0303
:1016100010919E0320919F033091A0036B017C01E8
:10162000C01AD10AE20AF30A9701860141E1C41601
:1016300047E2D406E104F10408F442C020919C037F
:1016400031E0320F30939C0320FF02C017E001C04D
:1016500010E060939D0370939E0380939F0390938B
:10166000A00363E070E084E094E00E94020161E086
:1016700070E084E094E00E94020107E0010F812FF6
:1016800090E0EC01CC0FDD1FC35FDE4F68817981F4
:10169000672F772763707727880F991F880F991F07
:1016A000682B792B84E094E00E94FA0068817981AC
:1016B000772784E094E00E94FA001F5F1013DFCFC9
:1016C000CDB7DEB7E8E00C94422125B190E0FC01F3
:1016D000EE0FFF1FE80FF91FE45FFC4F8081282BFE
:1016E00025B988B19181892B88B98BB19281892BD9
:1016F0008BB9089585B190910903892385B988B183
:1017000090910A03892388B98BB190910B038923A7
:101710008BB908951F920F920FB60F9211242F9339
:101720003F934F935F936F937F938F939F93AF9369
:10173000BF93CF93EF93FF93C0916803809106010D
:10174000C81708F03EC0809107039091080390935A
:10175000870080938600EC2FF0E0EE0FFF1FE35F21
:10176000FE4F808191810E94D902880F991F90932A
:101770000803809307038091070390910803209149
:10178000070130910801281B390B30930801209381
:1017900007018091F2039091F303880F991F281796
:1017A000390720F490930801809307018091660324
:1017B000811142C08091EA0380FF41C0C830E0F54A
:1017C0003EC0809107039091080390938700809317
:1017D00086008091070190910801909308038093FF
:1017E000070380916603882319F08FEF9FEF06C0EF
:1017F0008091070390910803885592409093890047
:101800008093880080E49CE990930801809307010D
:1018100080918400909185008097D0F30E947A0B8C
:1018200080916703811105C08091060181500E945B
:10183000650B1092680327C08FEF9FEF06C0809161
:1018400007039091080388559240909389008093F4
:10185000880080918400909185008097D0F30E9449
:101860007A0B80916703811104C080916803811114
:1018700006C0809168038F5F8093680304C0815025
:101880000E94650BF6CFFF91EF91CF91BF91AF9181
:101890009F918F917F916F915F914F913F912F9188
:1018A0000F900FBE0F901F90189524E0829FC001EB
:1018B00011248C30910538F0853F23E0920728F001
:1018C00084EF93E008958CE090E00895CF93DF9348
:1018D000C091EB03C03390F48C2F807339F08031CA
:1018E00041F4809169038295807F05C080916E03E9
:1018F00002C080916F03CF70D0E015C0CF33E0F409
:10190000CF70D0E0809169038295807F0E94550C52
:10191000DE01AA0FBB1FA35FBE4F11969C938E934F
:10192000219680916F030E94550CFE01EE0FFF1F60
:10193000E35FFE4F91838083DF91CF910895809183
:101940006A0390916B039F770E94FA028093690368
:101950008F3029F480916F038695805804C099E0F8
:10196000899F802D112480936E03F8940E94660C49
:1019700078948091DF038132E1F480916E039FEFD0
:10198000980F9E3F78F08091B0008F7D8093B000DB
:1019900061E080916E03811101C060E083E00E94EC
:1019A000541C08958093B4008091B00080628093AD
:1019B000B0000895FF920F931F93CF93DF930DED27
:1019C00013E0C0E0D0E0B3E0FB2E8C2FD801ED9106
:1019D0008D019E2F907F9031F1F4EF70F0E0EE0FCB
:1019E000FF1FE35FFE4F208131816F2D0E94BB20DE
:1019F000E92FF0E0EE0FFF1FE257FD4F61E080811D
:101A000091818217930708F060E0FE01E456FD4FD4
:101A100080810E94541C2196C630D105B1F6CDB705
:101A2000DEB7E5E00C9445210F931F93CF93DF932E
:101A300005E413E0C0E0D0E02091EB03822F8F702B
:101A400090E0C817D907E9F00196C817D90711F433
:101A50002033B8F4F801808191819F70892B79F04F
:101A6000F894F801808191819F700E94AE02FE017E
:101A7000EE0FFF1FE35FFE4F9183808378940E94F7
:101A8000DA0C21960E5F1F4FC031D105A9F6DF9108
:101A9000CF911F910F910895FF920F931F93CF93B2
:101AA000DF9383EB93E00E94A6018093060190915F
:101AB000EB03292F2F70281304C081E0820F80933D
:101AC000060190539F3060F44091060130E0842F6E
:101AD00090E001972817390719F44F5F40930601EA
:101AE00080910601813118F080E180930601EEE0DB
:101AF000F3E0DF0112971C92DF0111971C92108214
:101B0000339683E0E032F807A1F74FEF3FEFA4EA06
:101B1000B2E00DED13E02FEFE80189918E018031E5
:101B2000F8F490E0FD0132976081FC01EE0FFF1F99
:101B3000E80FF91FE45FFC4F8081862B8083CD0185
:101B40000197EC0158818181852B81839C91828151
:101B5000892B8283609550959095292335234623C0
:101B60001396D3E0033E1D07B9F640930903309363
:101B70000A0320930B03CCE9D2E00DED13E0F12C26
:101B8000F80181918F01823230F08632B8F08632CE
:101B900011F460E010C0F4E0FF1204C08091C100B5
:101BA0008F7E06C085E0F81205C08091C100877F56
:101BB0008093C10061E088810E941B1CF3942196F0
:101BC000E6E0FE12DDCF8091DD03803231F461E08A
:101BD00089E00E94541C82E801C082E0809380006A
:101BE00081E080936703809366038091DF038132F5
:101BF00011F08732D9F461E083E00E941B1C60E0A1
:101C000083E00E94541C8091DF03813231F481E033
:101C10008093B0008093B10009C082E08093B0004F
:101C200085E08093B1008EE38093B3008AE18093D6
:101C300081008FEF9FEF909389008093880080ED63
:101C400097E0909387008093860080E49CE99093CE
:101C50000801809307019093080380930703109273
:101C6000680380916F00816080936F008091EA0328
:101C700083FF0DC080914503909146039F70892B8F
:101C800031F00E94140D1092660310926703CDB7D5
:101C9000DEB7E5E00C9445219091DF03973259F4CB
:101CA000882321F08091B000806103C08091B00052
:101CB0008F7E8093B0000895A2E2B0E0E2E6FEE0FD
:101CC0000C941C216B017C010E94571B4B015C0191
:101CD00081E00E94600483E08093B0030E945E056F
:101CE00064EC71E084E094E00E94251D7BE1272EE6
:101CF000E0E53E2EF7E47F2EA6E44A2EB5E55B2E06
:101D0000C114D104E104F10469F00E94571B681961
:101D100079098A099B096C157D058E059F0510F0D0
:101D200080E0D5C08091B003843051F762ED71E05E
:101D300084E094E00E94251D8FE70E9447030E94E3
:101D40005A038AA3823601F503EB13E00E945A037B
:101D5000D8018D938D01B3E00C3D1B07B9F780913D
:101D6000B303883309F0ADC06BED71E084E094E01B
:101D70000E94251D82E48AA361E0CE0182960E9422
:101D8000BD05429A81E0A3C0803741F0893611F544
:101D900081E00E94750889E4898304C03982C12CDE
:101DA000D12C76019091AF038091EA03992311F031
:101DB000806801C08F778093EA03ECEDF3E0DE01E9
:101DC0001296822D01900D928A95E1F76CE1CE0179
:101DD000019675C08437E1F4E4E5E98383E08A8302
:101DE00088E88B8386E08C838CE08D8388E1EDE24C
:101DF000F1E0DE01169601900D928A95E1F76DE112
:101E0000CE0101960E94BD05C12CD12C760159C08E
:101E1000853789F40CED13E00E945A03D8018D93A5
:101E20008D01B3E0073F1B07B9F761E080E00E9436
:101E3000C7075AA241C08636B9F44982E5E4F3E007
:101E4000AE014D5F5F4F208131813296CA0101970B
:101E5000DC013C93DA012C934E5F5F4FB3E0E53633
:101E6000FB0789F761E2B3CF8736C9F405E413E0D5
:101E70000E945A03682E0E945A03262D30E0322F0A
:101E80002227280F311DF801219331938F01F3E0B0
:101E900005361F0769F77AA20E9461080DC08734D2
:101EA00081F4E5E4F3E01192119283E0E536F8075E
:101EB000D1F70E9461087AA261E0CE0182960E9469
:101EC000BD0583E08093B0030E943B0519CFA29625
:101ED000E2E10C9438211F93CF93DF93C82FD62FC4
:101EE00061E00E941B1C61E08C2F0E94541C61E089
:101EF0008D2F0E94541C8AE090E00E94AC1B8D2F15
:101F00000E94871C892B71F060E08C2F0E94541C6A
:101F10008AE090E00E94AC1B8D2F0E94871C11E08C
:101F2000892B09F010E060E08C2F0E941B1C60E000
:101F30008C2F0E94541C60E08D2F0E94541C812F16
:101F4000DF91CF911F91089580E48093BA001092A1
:101F5000BD008DE990E09093A8038093A7031092B1
:101F6000420315E004E0C2E0FC2E80914203813080
:101F700039F480E00E946004F09242034398F5CF68
:101F8000C0914203C33061F44298809184030E945F
:101F90008203C093B0030E943B0500934203E5CF48
:101FA00080914203843009F78091B0038430E9F6D0
:101FB0008FE70E944703C2EFD2E0E091DB03E770B6
:101FC000F0E0EC56FD4F808190E09E01225F3240B0
:101FD0002817390724F40E945A038993EECF1093EF
:101FE0004203429AC2CFAAE2B0E0E9EFFFE00C94CC
:101FF0002B211FEF198389E2E3EBF3E0DE01129658
:1020000001900D928A95E1F721E04AE2BE016F5FEF
:102010007F4F80E20E94520A81110EC021E041E010
:10202000BE016F5F7F4F80E20E94A70A811104C04A
:1020300082E08093420302C01093420380914203E6
:10204000823051F00E94571B60933E0370933F0310
:102050008093400390934103AA96E3E00C944721B8
:10206000A1E0B0E0E6E3F0E10C942C218091420382
:102070008230D9F480918403805A898321E041E041
:10208000BE016F5F7F4F80E20E94520A882369F091
:102090008FEF809342030E94571B60933E0370931F
:1020A0003F0380934003909341032196E2E00C9418
:1020B0004821A1E0B0E0EFE5F0E10C942C21809103
:1020C00042038230D1F421E041E0BE016F5F7F4FD7
:1020D00080E20E94A70A882371F08FEF8093420369
:1020E0000E94571B60933E0370933F03809340030D
:1020F0009093410302C0898101C08FEF2196E2E0F5
:102100000C944821A2E2B0E0E8E8F0E10C941C2134
:102110009E012F5F3F4F80E1D9011D928A95E9F71B
:1021200066EE71E084E094E029A33AA30E94251DA5
:102130000E945E051D8A1E8A1F8A188E312C212C52
:1021400000E0812C912C540180E4482E81EE582E21
:102150008DE9682E88E1782E90E5C92E93ECD92E72
:10216000E12CF12C84EF91E0A0E0B0E08D8F9E8F08
:10217000AF8FB8A380EC91EDA8E9BBE1898F9A8F6E
:10218000AB8FBC8F80E491EEADE9B8E1898B9A8B7F
:10219000AB8BBC8B84E094E00E94F11D892B09F489
:1021A000E1C084E094E00E941E1E9C0133272C3283
:1021B000310509F442C0ACF42332310509F0ABC05B
:1021C00019821A821B821C821D821E821F8218861F
:1021D00019861A861B861C861D861E861F86188AEF
:1021E00060C02434310529F02335310509F4B2C02B
:1021F00092C064E484E094E00E94091D2AE030E08B
:1022000040E451EE6DE978E184E094E00E94851DA0
:102210006CE284E094E00E94091D2AE030E040EC8A
:1022200051ED68E97BE184E094E00E94851D6CE259
:1022300084E094E00E94371DADCF0F5F043009F0B9
:10224000A9CF29813A814B815C81A8EEB3E00E943D
:102250009820698B7A8B8B8B9C8B2D813E814F8153
:1022600058850E949820698F7A8F8B8F9C8F298543
:102270003A854B855C852D8F3E8F4F8F58A32D85DA
:102280003E854F8558890E9498206B017C01603201
:102290003EE473078105910530F462E38CE10E940E
:1022A0006F0300E077CF603345E774078105910540
:1022B00010F462E2F3CF60345CE9750781059105A3
:1022C00010F466E2EBCF80E5C81683ECD806E10493
:1022D000F10410F462E1E2CF90E6C9169AEED90655
:1022E000E104F10410F465E1D9CFA0E7CA16A1E139
:1022F000DA06A1E0EA06F10410F461E0CFCFB0EA1B
:10230000CB16B6E8DB06B1E0EB06F10410F463E0AF
:10231000C5CF65E0C3CF10ED180F1A3008F03ACFE3
:10232000E1E0F0E0EC0FFD1F24E0029FE00DF11D65
:1023300011242081318142815381AAE0B0E00E94C2
:102340009820610F711D811D911D608371838283AF
:10235000938320CF49885A886B887C88812C912C64
:10236000540118CF81149104A104B10489F4C3016C
:10237000B2010E94F50361E070E080E090E00E940D
:10238000861B1D8A1E8A1F8A188E312C22242A94AD
:102390008D8D9E8DAF8DB8A188169906AA06BB06B5
:1023A000D0F40E9498032D893E894F89588D280FBB
:1023B000311D411D511D2D8B3E8B4F8B588F381673
:1023C00008F4382E821508F4282E3FEF831A930A5A
:1023D000A30AB30A56C0C301B20128EE33E040E0BD
:1023E00050E00E94DB20BA01A9012AE030E084E03D
:1023F00094E00E94D31D6CE284E094E00E94091DE9
:102400004AE050E0632D84E094E00E94E21D6CE21B
:1024100084E094E00E94091D6D897E898F89988DE2
:10242000A50194010E94DB20BA01A9012AE030E055
:1024300084E094E00E94D31D6CE284E094E00E946A
:10244000091D4AE050E0622D84E094E00E94E21D04
:102450006CE284E094E00E94371D4C0C5D1C6E1C05
:102460007F1C898D9A8DAB8DBC8D84159505A60535
:10247000B70520F449885A886B887C88812C912C78
:10248000540129893A894B895C89283E33404105AA
:10249000510509F07FCEA296E2E10C943821A1E02B
:1024A000B0E0E5E5F2E10C942C2180E00E948C0183
:1024B00061E080E10E941B1C61E081E10E941B1C25
:1024C0000E94630160E080E00E941B1C61E081E0EB
:1024D0000E941B1C40E052EC61E070E084E094E05C
:1024E0000E94391F0E94B3080E94660863EF71E0E2
:1024F00084E094E00E94061D88E893E00E94620751
:102500006AE072E084E094E00E94061D4AE050E038
:1025100068E070E084E094E00E94BB1D0E947801B6
:102520007894439A63E183E00E946B0F882329F03B
:10253000439842980E948210FBCF62E189E00E949A
:102540006B0F811104C00E944F08811119C06DE406
:1025500072E084E094E00E94061D60E070E0CB0130
:102560000E945C0E882349F00E945C0862E172E0E0
:1025700084E094E00E94251D429A0E944C0D10C0F8
:102580000E944C0D8091DE03823209F0C6C080911A
:10259000E003833209F0C1C08091EA0381FDC3C02A
:1025A0008091DE03823231F58091E003833211F5B0
:1025B00081E00E94BD088091EA0382FF08C06DE2BD
:1025C00072E084E094E00E94251D0E94A40F64E163
:1025D00070E080E090E00E94861B21E041E0BE01B7
:1025E0006F5F7F4F80E20E94A70A811103C081E0E4
:1025F0008093420368E372E084E094E00E94061D49
:102600008FE00E948C0180E00E946004109284039D
:1026100080E00E94820380E0883170F08093C602DF
:1026200083E08093B0030E945E058091420388237B
:1026300071F00E94F30F0BC021E0280FE82FF0E0AB
:10264000ED54FC4F9785992349F3822FE5CF809174
:10265000E203982F9D7F983229F440E052EC61E02C
:1026600070E023C0893251F42EE240EA56E861E07E
:1026700070E084E094E00E94BA1F1BC08091DB03ED
:102680008871803129F440E855E260E070E00DC0C7
:102690004091B4035091B5036091B6037091B703B4
:1026A0004A3051056105710570F384E094E00E94A1
:1026B000391F84E094E00E94F11D892B29F084E009
:1026C00094E00E941E1EF5CF8091E103843229F030
:1026D0008091C1008F7E8093C1008091E20385329A
:1026E00041F08852833028F08091C100877F809329
:1026F000C1001092C8021092C702109244030E94B7
:10270000631B609380037093810380938203909393
:1027100083032196E2E00C9448218091EA038B7FA9
:102720008093EA0339CF82FD3BCF64EF71E080E014
:1027300090E00E945C0E882309F432CF0E945C086E
:1027400062E172E084E094E00E94251D0E944C0D3D
:10275000429A26CFCF93DF9384E094E00E94F11D4C
:10276000892BE9F0C091C702D0E0CE0101968F71AC
:1027700099272091C80230E08217930781F084E006
:1027800094E00E941E1EC753DD4F88838091C702CC
:1027900090E001968F7199278093C702DDCFDF917A
:1027A000CF910895A0E0B0E0E8EDF3E10C9426218C
:1027B000D82FC62F0E94631B00919D0310919E038A
:1027C00020919F033091A0036B017C01C01AD10AB4
:1027D000E20AF30A9701860141E1C41647E2D406F2
:1027E000E104F10408F4D1C160939D0370939E034A
:1027F00080939F039093A00380910D0190910E010F
:10280000880F991F80938503892F877020918603F5
:10281000287F282B2093860380910F01909110012F
:10282000880F991F382F330F330F330F2770232B47
:1028300020938603282F2295269527708091870361
:10284000807C9770990F990F990F822B892B809319
:1028500087032091110130911201220F331F922F13
:102860009295990F990F907C8F73892B8093870392
:10287000932F9295990F990F907C822F869586952C
:10288000892B8093880332FB882780F92091890364
:102890002E7F282B2093890380911301909114019E
:1028A000880F991F382F330F2170232B2093890312
:1028B000382F331F3327331F20918A03207F892F1E
:1028C0008770880F232B282B20938A038091150172
:1028D00090911601880F991F382F3295307F2F70F5
:1028E000232B20938A03382F32953F7020918B033E
:1028F0002078892F87708295807F232B282B209327
:102900008B038091170190911801880F991F2F77E1
:1029100020938B03292F2795222727958695822B95
:1029200080938C03892F8695837020918D032C7F53
:10293000282B20938D038091190190911A01880F03
:10294000991F382F330F330F2370232B20938D03C0
:10295000382F329536953695337020918E03207E30
:10296000892F8770880F880F232B282B20938E03A5
:1029700080911B0190911C01880F991F382F32956F
:10298000330F307E2F71232B20938E039295990F56
:10299000907E869586958695892B80938F0380916E
:1029A0001D0190911E01880F991F80939003892F1C
:1029B000877020919103287F282B20939103809189
:1029C0001F0190912001880F991F382F330F330F6B
:1029D000330F2770232B20939103282F22952695C0
:1029E000277080919203807C9770990F990F990FAF
:1029F000822B892B80939203209121013091220117
:102A0000220F331F922F9295990F990F907C8F73FD
:102A1000892B80939203932F9295990F990F907C15
:102A2000822F86958695892B8093930332FB882786
:102A300080F9209194032E7F282B2093940380917A
:102A4000230190912401880F991F382F330F217093
:102A5000232B20939403382F331F3327331F2091C8
:102A60009503207F892F8770880F232B282B209395
:102A700095038091250190912601880F991F382F89
:102A80003295307F2F70232B20939503382F32956A
:102A90003F70209196032078892F87708295807FE0
:102AA000232B282B209396038091270190912801B6
:102AB000880F991F2F7720939603292F2795222778
:102AC00027958695822B8093970396959370809196
:102AD00098038C7F892B8093980320912901309152
:102AE0002A01220F331F922F990F990F8370892B80
:102AF00080939803229526952695237080919903BB
:102B0000807E932F9770990F990F822B892B80933A
:102B1000990320912B0130912C01220F331F922F0A
:102B20009295990F907E8F71892B80939903832FB3
:102B30008295880F807E269526952695282B2093B2
:102B40009A03DD2311F088E001C080E0CC2311F06E
:102B500094E001C090E0892B80939B036FE070E0CC
:102B600084E094E00E940201C5E8D3E0699184E02A
:102B700094E00E944B1E83E0CC39D807B9F760E09F
:102B800070E084E094E00E940201CDB7DEB7E8E097
:102B90000C944221CF93C82F682F84E094E00E94C8
:102BA0004B1E8C2F0E940A01CF910895A0E0B0E047
:102BB000ECEDF5E10C942621C82F0E94631B0091D7
:102BC0009D0310919E0320919F033091A0036B0100
:102BD0007C01C01AD10AE20AF30A9701860141E199
:102BE000C41647E2D406E104F10408F445C060933A
:102BF0009D0370939E0380939F039093A003109274
:102C0000B2031092B10388EA0E94CA15CC2311F0D6
:102C100081E801C081E00E94CA1580E10E94CA15C6
:102C200000E010E0F801EE0FFF1FE35FFE4F808130
:102C300091810E94D902EC01B3E0CC0FDD1FBA955F
:102C4000E1F78D2F0E94CA158C2F0E94CA150F5FC5
:102C50001F4F0031110531F76091B20370E084E03D
:102C600094E00E94FA006091B1037091B20377275B
:102C700084E094E00E94FA00CDB7DEB7E8E00C945F
:102C80004221AAE1B0E0E7E4F6E10C941E210E94A3
:102C90009B008CE00E94690381110BC066E872E022
:102CA00084E094E00E94251D80E00E9460040E9460
:102CB0005E050E94AA130E94631B0E94591091E0B6
:102CC000853009F090E01FEF8091B003843009F463
:102CD00006C2911104C284C00E949C0390936D03AC
:102CE00080936C03429AC0928003D0928103E09259
:102CF0008203F092830310924303109274031092A4
:102D00007503109276031092770380916A03909175
:102D10006B03880F991F816090936B0380936A0304
:102D2000439880E00E944C0E8091F202982F9E738F
:102D300009F02CC2F8948091DB0343EF52E06DE080
:102D400071E087700E9428020E94660C789490912E
:102D5000F20280913C0390FF13C2811124C095E4DC
:102D6000E92E93E0F92E00E010E0F70180819181D7
:102D700094FD0CC0F801EE0FFF1FE35FFE4F808152
:102D800091810E94D902D7018D939C930F5F1F4FB1
:102D9000B2E0EB0EF11C0031110539F70E94610819
:102DA00081E080933C0380914403811103C081E062
:102DB0008093440310926503109267031092660398
:102DC0008091DB03887109F009C20E94DA0C83E06C
:102DD0008093B0030E943B0581E080933D034298BD
:102DE0000E94631B4B015C010E94571B6B017C011D
:102DF00080914303823008F063C04090800350907C
:102E00008103609082037090830380917C03909192
:102E10007D03A0917E03B0917F0384159505A605DF
:102E2000B70509F44DC083EB93E00E94B6016C5DD9
:102E30007540810991099501840104191509260934
:102E400037096017710782079307D0F540927C031A
:102E500050927D0360927E0370927F030E949803DC
:102E6000282F809370038091710390917203820FD9
:102E7000911D9093720380937103609173036F5F50
:102E8000609373036930E0F070E00E94C720709394
:102E900072036093710380916F03E3E08E9F600D76
:102EA000711D1124769567957695679560936F03EC
:102EB0000E949F0C10927203109271031092730380
:102EC000809144030091C602882351F1109143037D
:102ED000101708F029C24090800350908103609041
:102EE000820370908303A5019401241935094609D2
:102EF00057092F8B388F498F5A8F83EB93E00E94AD
:102F0000B60168517C4F8F4F9F4F2F89388D498D67
:102F10005A8D621773078407950708F4CCC104C261
:102F20008091800390918103A0918203B0918303EB
:102F300075016401C81AD90AEA0AFB0A83EB93E017
:102F40000E94B6019B01AC01A02FB0E00E94982026
:102F50006C157D058E059F0558F480928003909234
:102F60008103A0928203B092830381E080933D03AA
:102F700080916603811116C08091E203883219F4B2
:102F80000E94FE0A0FC0893239F460914303809198
:102F900065030E94D21306C08A3221F48091650332
:102FA0000E94D61580913D03882309F472C0E091F8
:102FB0008403EF5FE0938403E83131F0F0E0ED54F7
:102FC000FC4F8785811102C0109284038091EC032D
:102FD0009091ED03A091EE03B091EF03892B8A2B22
:102FE0008B2B09F44EC08091740390917503A091CE
:102FF0007603B0917703892B8A2B8B2B09F441C080
:103000000E944E06082F10E02091090130910A011C
:1030100036952795369527952C5E3F4F201731071B
:1030200070F40E94571B68517C4F8F4F9F4F6093E5
:103030007403709375038093760390937703C801AC
:10304000880F991F880F991F4091090150910A011B
:103050009A01220F331F240F351F820F931F96955D
:1030600087959695879590930A01809309016091C1
:10307000B8037091B9038091BA039091BB030E9489
:10308000F503809184030E9482030E943010109205
:103090003D03809142038F3F09F041C20E94571BBC
:1030A00000913E0310913F03209140033091410372
:1030B000601B710B820B930B693E73408105910578
:1030C00008F42DC20E94571B60933E0370933F0388
:1030D00080934003909341030E94F30F20C20E940B
:1030E000631B6B017C018091B0038430D1F48FE7C6
:1030F0000E94470302EF12E0E091DB03E770F0E08B
:10310000EC56FD4F808190E09801225F32402817F5
:1031100039070CF0E1CD0E945A03D8018D938D013F
:10312000EBCFE091DB03E770F0E0EC56FD4F408120
:103130004F5F21E0BE016F5F7F4F80E20E94A70AD0
:10314000882371F0109342030E94571B60933E0343
:1031500070933F03809340039093410390E0B4CD7C
:10316000E091DB03E770F0E0EC56FD4F408150E06A
:10317000BE016E5F7F4F82EF92E00E945921B3CD76
:10318000882309F410CE10923C030DCE982F98732B
:10319000983309F008CE9091E902892787FF03CE82
:1031A00090589093E9028091E203853209F0FBCDBB
:1031B00010E0212F30E08091F202877090E08217BA
:1031C00093070CF4F0CD1F5FE12FF0E0EE50FD4FC0
:1031D000608184E094E00E944B1EEBCF8091E90275
:1031E0009091F202982796FD5AC0807C90E489273E
:1031F0008093E9028091C8023091C7028317D1F011
:10320000EAEEF2E020E02F5F90E0DC01A753BD4F33
:103210004C91419301968F719927283011F08313B7
:10322000F2CF8093C802295C8091E902282B209379
:10323000E90235C0809170038093EA028091DE0339
:10324000863251F482E10E94B01C95958795959540
:1032500087958093EB0202C01092EB028091E0030D
:10326000863251F483E10E94B01C9595879595951F
:1032700087958093EC0202C01092EC0280916C035F
:1032800090916D039093ED028093EE0280916A031A
:1032900090916B039F770E94FA028093EF0269E09E
:1032A00089EE92E00E9476050E94E50581118DCDA0
:1032B0000E94AA13F9CF80916A0390916B03880F43
:1032C000991F90936B0380936A0381E080933D0381
:1032D000111110C0C0927803D0927903E0927A0362
:1032E000F0927B0310927403109275031092760390
:1032F000109277031F5F1093430383EB93E00E94C8
:10330000B601640D751D861D971D60938003709333
:1033100081038093820390938303439A81E00E9408
:103320004C0E0E949F0C03C0101709F4A7C0809197
:103330004303882309F41CCE8091F4038823D9F039
:1033400090916503911117C04091780350917903D2
:1033500060917A0370917B0346015701841A950AA4
:10336000A60AB70A90E00E942301681579058A052C
:103370009B0508F4B5C08091F6038823D9F090919D
:103380006703911117C040917803509179036091C0
:103390007A0370917B0346015701841A950AA60AA5
:1033A000B70A90E00E942301681579058A059B05FC
:1033B00008F4ADC08091F5038823D9F0909166039D
:1033C000911117C0409178035091790360917A036D
:1033D00070917B0346015701841A950AA60AB70A21
:1033E00090E00E942301681579058A059B0508F481
:1033F00092C08091EC039091ED03A091EE03B09107
:10340000EF03892B8A2B8B2B09F4B2CD80917403A7
:1034100090917503A0917603B09177030097A10571
:10342000B10509F4A5CDC81AD90AEA0AFB0AF7FCC6
:103430009FCD8091EA03829581700E94910680E081
:103440000E9460040E943B050E94571B6B017C0197
:103450002091F10330E0A8EEB3E00E948920C60E6F
:10346000D71EE81EF91E6894C0F8C0927403D0926B
:103470007503E0927603F09277037ACD8091800312
:1034800090918103A0918203B091830324013501BF
:10349000481A590A6A0A7B0A83EB93E00E94B60134
:1034A0009B01AC01A12FB0E00E9498206415750526
:1034B0008605970508F03BCF10926B0310926A03C4
:1034C00081E080933D0310926F030E949F0C8092D5
:1034D000800390928103A0928203B092830327CF4E
:1034E00081E0809365030E94140D8091F0030E9497
:1034F00048016C0D7D1D8E1D9F1D616060937403DE
:1035000070937503809376039093770334CF81E0B3
:10351000809367034FCF81E0809366036ACF6A96FA
:10352000E0E10C943A218230E8F4E82FF0E0EE0F6D
:10353000FF1FE950FC4F71836083813041F080911F
:1035400069008C7F842B80936900E89A08958091AC
:103550006900440F551F440F551F837F842B8093B0
:103560006900E99A08951F920F920FB60F921124E5
:103570002F933F934F935F936F937F938F939F937B
:10358000AF93BF93EF93FF938091F7039091F8036C
:10359000892B29F0E091F703F091F8030995FF9149
:1035A000EF91BF91AF919F918F917F916F915F91BB
:1035B0004F913F912F910F900FBE0F901F90189534
:1035C0001F920F920FB60F9211242F933F934F9398
:1035D0005F936F937F938F939F93AF93BF93EF937B
:1035E000FF938091F9039091FA03892B29F0E091E0
:1035F000F903F091FA030995FF91EF91BF91AF9113
:103600009F918F917F916F915F914F913F912F91FA
:103610000F900FBE0F901F9018951F920F920FB62C
:103620000F9211242F933F938F939F93AF93BF9348
:103630008091FC039091FD03A091FE03B091FF03E4
:103640003091FB0323E0230F2D3720F40196A11DB9
:10365000B11D05C026E8230F0296A11DB11D2093C0
:10366000FB038093FC039093FD03A093FE03B093B0
:10367000FF038091000490910104A0910204B09195
:1036800003040196A11DB11D8093000490930104D1
:10369000A0930204B0930304BF91AF919F918F91C7
:1036A0003F912F910F900FBE0F901F9018952FB73D
:1036B000F8946091FC037091FD038091FE0390915A
:1036C000FF032FBF08953FB7F894809100049091B5
:1036D0000104A0910204B091030426B5A89B05C083
:1036E0002F3F19F00196A11DB11D3FBF6627782F0E
:1036F000892F9A2F620F711D811D911D42E0660F67
:10370000771F881F991F4A95D1F70895CF92DF92AE
:10371000EF92FF92CF93DF936B017C010E94631BBA
:10372000EB01C114D104E104F10479F00E94631BA0
:103730006C1B7D0B683E7340A0F381E0C81AD10872
:10374000E108F108C851DC4FECCFDF91CF91FF9039
:10375000EF90DF90CF9008950197009739F0880F90
:10376000991F880F991F02970197F1F70895789490
:1037700084B5826084BD84B5816084BD85B5826076
:1037800085BD85B5816085BDEEE6F0E08081816014
:103790008083E1E8F0E01082808182608083808114
:1037A00081608083E0E8F0E0808181608083E1EBEC
:1037B000F0E0808184608083E0EBF0E080818160D4
:1037C0008083EAE7F0E0808184608083808182608A
:1037D0008083808181608083808180688083109273
:1037E000C1000895833081F028F4813099F082304F
:1037F000A1F008958630A9F08730B9F08430D1F473
:10380000809180008F7D03C0809180008F778093AE
:103810008000089584B58F7702C084B58F7D84BD04
:1038200008958091B0008F7703C08091B0008F7DA4
:103830008093B0000895CF93DF9390E0FC01E458AB
:10384000FF4F2491FC01E057FF4F8491882349F1F9
:1038500090E0880F991FFC01E854FF4FA591B491A7
:1038600082559F4FFC01C591D4919FB7611108C04B
:10387000F8948C91209582238C93888182230AC0AE
:10388000623051F4F8948C91322F309583238C93CD
:103890008881822B888304C0F8948C91822B8C932E
:1038A0009FBFDF91CF910895A1E0B0E0EAE5FCE190
:1038B0000C942A21282F30E0F901E859FF4F849118
:1038C000F901E458FF4F1491F901E057FF4F0491BB
:1038D0000023C9F0882321F069830E94F21B6981CB
:1038E000E02FF0E0EE0FFF1FE255FF4FA591B491DE
:1038F0009FB7F8948C91611103C01095812301C08A
:10390000812B8C939FBF2196E4E00C944621CF93AA
:10391000DF93282F30E0F901E859FF4F8491F90136
:10392000E458FF4FD491F901E057FF4FC491CC23E5
:1039300091F081110E94F21BEC2FF0E0EE0FFF1FBF
:10394000EC55FF4FA591B4912C912D2381E090E08F
:1039500021F480E002C080E090E0DF91CF910895F3
:103960008E3008F08E5087702091B70190E4299F27
:1039700090011124822B80937C0080917A008064D6
:1039800080937A0080917A0086FDFCCF8091780048
:103990002091790090E0922B0895A0E0B0E0E3ED53
:1039A000FCE10C9426216C017A01EB01E60EF71E76
:1039B00000E010E0CE15DF0561F06991D601ED91D0
:1039C000FC910190F081E02DC6010995080F191FA7
:1039D000F1CFC801CDB7DEB7E8E00C944221611504
:1039E000710589F0DB010D900020E9F7AD01415030
:1039F0005109461B570BDC01ED91FC910280F381CC
:103A0000E02D0995089580E090E008950E94EF1C54
:103A10000895DC01ED91FC910190F081E02D099574
:103A200008950F931F93CF93DF93EC016DE00E94F5
:103A3000091D8C016AE0CE010E94091D800F911FB3
:103A4000DF91CF911F910F9108950F931F93CF9303
:103A5000DF93EC010E94EF1C8C01CE010E94111D2E
:103A6000800F911FDF91CF911F910F9108950F93B8
:103A70001F93CF93DF93EC010E94091D8C01CE01AF
:103A80000E94111D800F911FDF91CF911F910F9107
:103A90000895A1E2B0E0EFE4FDE10C9422217C0165
:103AA000C42EE52FCB01D22E19A221E02D1510F046
:103AB0002AE0D22E8E010F5D1F4F8D2C912CA12C50
:103AC000B12C6C2D7E2FA50194010E94DB208C2D42
:103AD000D29E80191124015011098A3010F4805DA2
:103AE00001C0895CF801808321153105410551052C
:103AF00021F0C22EE32FCA01E4CFB801C7010E9412
:103B0000EF1CA196ECE00C943E21A0E0B0E0EBE8C5
:103B1000FDE10C942621EC016A017B0121153105A0
:103B200041F4E881F9810190F081E02D642F09953D
:103B30001DC02A303105A9F477FF12C06DE20E9442
:103B4000091D8C0144275527BA014C195D096E09DE
:103B50007F092AE0CE010E94491D800F911F06C0F7
:103B60002AE0B701A601CE010E94491DCDB7DEB7FC
:103B7000E8E00C9442210F931F93CF93DF93EC0165
:103B80009A01AB01662757FD6095762F0E94851D2F
:103B90008C01CE010E94111D800F911FDF91CF91EA
:103BA0001F910F9108952115310549F4DC01ED9124
:103BB000FC910190F081E02D642F099508950E94F9
:103BC000491D08959A01462F50E060E070E00E9480
:103BD000D31D08959A01AB0160E070E00E94D31DEF
:103BE0000895FC0124853585F901E05CFF4F808153
:103BF0009181F901EE5BFF4F20813181821B930B94
:103C00008F7399270895FC0184859585FC01E05CFC
:103C1000FF4F40815181FC01EE5BFF4F20813181DC
:103C20004217530741F00190F081E02DE80FF91F92
:103C3000808190E008958FEF9FEF0895FC018485C7
:103C40009585FC01E05CFF4F40815181FC01EE5BFA
:103C5000FF4F208131814217530779F0A081B18154
:103C6000A80FB91F8C91208131812F5F3F4F2F7397
:103C700033273183208390E008958FEF9FEF0895DD
:103C8000FC0181A1882329F0A489B5898C9186FF44
:103C9000FBCF11A20895CF93DF93FC0126853785D2
:103CA000D901A05CBF4F8D919C91119701968F73A4
:103CB0009927E901CE5BDF4F488159818417950729
:103CC000D9F30D90BC91A02DA20FB31F6C93A685C4
:103CD000B785A05CBF4F11969C938E93A689B78938
:103CE0002C9181E090E0078C02C0880F991F0A9404
:103CF000E2F7282B2C9381E081A30488F589E02D3D
:103D000080818064808381E090E0DF91CF9108958D
:103D100008951F920F920FB60F9211242F933F9385
:103D20004F938F939F93EF93FF938091C00082FDF9
:103D30001CC04091C6008091AA049091AB040196EA
:103D40008F7399272091AC043091AD0482179307AB
:103D500071F0E091AA04F091AB04E659FB4F408367
:103D60009093AB048093AA0402C08091C600FF9197
:103D7000EF919F918F914F913F912F910F900FBE97
:103D80000F901F90189584E094E00E94F11D892BFC
:103D900011F00E94881E08951F920F920FB60F9285
:103DA00011242F933F938F939F93EF93FF93209131
:103DB0006604309167048091680490916904281723
:103DC000390731F48091C1008F7D8093C10014C008
:103DD000E0916804F0916904EA5DFB4F20818091D5
:103DE00068049091690401968F73992790936904F0
:103DF000809368042093C600FF91EF919F918F916B
:103E00003F912F910F900FBE0F901F901895A0E03B
:103E1000B0E0EDE0FFE10C942221FC01138212825C
:103E200088EE93E0A0E0B0E084839583A683B78317
:103E300088EB92E0918380837587648757874687F4
:103E4000318B208B138B028BF58AE48AD78AC68A42
:103E5000B18EA08E938E828E8F85848F8889858F78
:103E60008989868F8A89878F8B8980A3ECE00C945F
:103E70003E21CF92DF92EF92FF92CF93DF93EC013E
:103E80006A017B01411581EE580761057105F9F062
:103E9000EC89FD8981E090E008A002C0880F991F9D
:103EA0000A94E2F7808360E079E08DE390E0A70177
:103EB00096010E94DB202150310941095109569594
:103EC000479537952795211580E1380798F0EC89BB
:103ED000FD89108260E874E88EE190E0A701960108
:103EE0000E94DB202150310941095109569547951F
:103EF00037952795E889F9893083EA89FB892083FA
:103F000019A2EE89FF89408181E090E09C010C8C30
:103F100002C0220F331F0A94E2F7422B4083EE893E
:103F2000FF8940819C010D8C02C0220F331F0A942F
:103F3000E2F7422B4083EE89FF8940819C010E8C81
:103F400002C0220F331F0A94E2F7422B4083EE890E
:103F5000FF8920810F8C02C0880F991F0A94E2F715
:103F6000809582238083DF91CF91FF90EF90DF9047
:103F7000CF900895BF92CF92DF92EF92FF92CF93AE
:103F8000DF93EC016A017B01B22E411581EE5807E7
:103F900061057105F9F0EC89FD8981E090E008A0E8
:103FA00002C0880F991F0A94E2F7808360E079E0ED
:103FB0008DE390E0A70196010E94DB20215031099A
:103FC000410951095695479537952795211580E167
:103FD000380798F0EC89FD89108260E874E88EE17A
:103FE00090E0A70196010E94DB2021503109410990
:103FF00051095695479537952795E889F989308372
:10400000EA89FB892083E88DF98DB082EE89FF89EA
:10401000408181E090E09C010C8C02C0220F331F94
:104020000A94E2F7422B4083EE89FF8940819C018C
:104030000D8C02C0220F331F0A94E2F7422B4083FB
:10404000EE89FF8940819C010E8C02C0220F331F34
:104050000A94E2F7422B4083EE89FF8920810F8C7E
:1040600002C0880F991F0A94E2F78095822380830B
:10407000DF91CF91FF90EF90DF90CF90BF900895A8
:104080008F929F92AF92BF92CF92DF92EF92FF9268
:104090000F931F9381E08F9385E08F9387E08F9339
:1040A00083E08F9384E08F93E6EC8E2E912CF2ECDC
:1040B000AF2EB12CA1ECCA2ED12CB0ECEB2EF12CF2
:1040C00004EC10E025EC30E046E254E06AE674E0EF
:1040D00084E094E00E94071F0F900F900F900F90C4
:1040E0000F901F910F91FF90EF90DF90CF90BF90B6
:1040F000AF909F908F9008950E94B71B0E944F121F
:10410000C3ECDEE10E9441162097E1F30E94C31E3A
:10411000F9CFA29FB001B39FC001A39F700D811D75
:104120001124911DB29F700D811D1124911D0895C0
:104130000E948920A59F900DB49F900DA49F800D93
:10414000911D11240895B7FF0C9498200E94982087
:10415000821B930B0895DB018F939F930E949820FD
:10416000BF91AF91A29F800D911DA39F900DB29F13
:10417000900D11240895991B79E004C0991F96179A
:1041800008F0961B881F7A95C9F780950895AA1B99
:10419000BB1B51E107C0AA1FBB1FA617B70710F032
:1041A000A61BB70B881F991F5A95A9F78095909564
:1041B000BC01CD010895A1E21A2EAA1BBB1BFD0173
:1041C0000DC0AA1FBB1FEE1FFF1FA217B307E407F6
:1041D000F50720F0A21BB30BE40BF50B661F771F4E
:1041E000881F991F1A9469F760957095809590952E
:1041F0009B01AC01BD01CF010895052E97FB1EF474
:1042000000940E94142157FD07D00E94DB2007FC78
:1042100003D04EF40C94142150954095309521957F
:104220003F4F4F4F5F4F08959095809570956195E2
:104230007F4F8F4F9F4F08952F923F924F925F92E3
:104240006F927F928F929F92AF92BF92CF92DF92A6
:10425000EF92FF920F931F93CF93DF93CDB7DEB70B
:10426000CA1BDB0B0FB6F894DEBF0FBECDBF09949F
:104270002A88398848885F846E847D848C849B84F6
:10428000AA84B984C884DF80EE80FD800C811B8104
:10429000AA81B981CE0FD11D0FB6F894DEBF0FBE33
:1042A000CDBFED010895EE0FFF1F0590F491E02DB5
:1042B0000994FB01DC0102C001900D924150504075
:1042C000D8F70895F999FECF92BD81BDF89A992744
:1042D00080B50895262FF999FECF1FBA92BD81BDF2
:1042E00020BD0FB6F894FA9AF99A0FBE0196089578
:0442F000F894FFCF70
:1042F4000000AE04200008409CFF00881300020068
:104304000200020002000200020002000200020099
:10431400020002000200020002000200020020016A
:10432400220126022102270323032604240525054E
:10433400280529052A8025000005400AA1204EA54C
:104344000020244EA52C2330C01200001A400AA1DC
:10435400204EA5001B1E27522C233080250000056B
:10436400400AA1204EA50020244EA52C2330004B4A
:10437400000006400AD0009D49007B289D492C235B
:104384003000E1000005400A4501D7DC03B81E0EE9
:10439400BF00232E48E801008A400A6001555502F7
:1043A400AD1E20000023C80154582074696D656F48
:1043B4007574210057616974696E672062696E645F
:1043C4000A00476F7420706B740A00646174612082
:1043D400676F6F640A007363616E6E6572206D6F40
:1043E4006465004F70656E4C52536E6720525820BE
:1043F4007374617274696E672000206F6E20485771
:10440400200053617665642062696E64206461747F
:104414006120746F20454550524F4D0A0049206178
:104424006D20736C61766500456E746572696E67A4
:10443400206E6F726D616C206D6F64650045455030
:10444400524F4D2064617461206E6F742076616CEC
:104454006964206F722062696E64206A756D707081
:104464006572207365742C20666F7263696E6720B1
:1044740062696E640A0052582068616E6700B20077
:10448400F4014C0300070B0C10111500091203135F
:1044940000010200000010000000080020000000DD
:1044A40001000002000000004B1ECD1CF11D1E1E69
:0444B400031E401E85
:107E00000F92CDB7DEB7112484B714BE81FFF1D035
:107E100082E08093C00088E18093C10086E0809377
:107E2000C20080E18093C4008EE0CDD088249924E4
:107E3000CC24C394F5E0DF2EE1E1EE2E73E0F72EC3
:107E4000B6D0082F813479F4B2D08983C2D0898129
:107E5000823811F481E005C0813811F485E001C059
:107E600083E09ED09AC0823411F484E103C085344B
:107E700019F485E0B6D091C0853561F498D0082F0B
:107E800010E095D090E0982E8824802A912A880CC2
:107E9000991C82C0863521F484E0A3D080E0E1CF34
:107EA000843609F04CC083D082D0A82E80D0B82E62
:107EB00000E011E07CD0F80181938F01AE16D1F77C
:107EC00088D0FB2DF53489F4E0E0F1E00BC0F9999E
:107ED000FECF92BC81BC0894811C911C819180BD15
:107EE000FA9AF99AEA1598F358C08B2D863409F05E
:107EF00054C0F401F7BEE89507B600FCFDCFF401CD
:107F0000A0E0B1E02C9130E011968C91119790E0B7
:107F1000982F8827822B932B12960C01C7BEE895C9
:107F20001124329681E0A038B80761F7F401D7BE7A
:107F3000E89507B600FCFDCFE7BEE8952EC0843774
:107F4000F1F435D034D0182F32D0B82E42D0FB2DDA
:107F5000F63421F4F40105914F010CC0FB2DF534EA
:107F600049F4F999FECF92BC81BC0894811C911C04
:107F7000F89A00B5802F14D0115049F70EC08537FC
:107F800039F427D08EE10CD085E90AD08FE069CF93
:107F9000813511F488E017D01CD080E101D050CF9A
:107FA0009091C00095FFFCCF8093C600089580910A
:107FB000C00087FFFCCF8091C00084FD01C0A89560
:107FC0008091C6000895E0E6F0E098E19083808318
:107FD0000895EDDF803219F088E0F5DFFFCF84E10E
:107FE000DFCF1F93182FE3DF1150E9F7F2DF1F9166
:0E7FF0000895282E80E0E7DFEE27FF27099492
:027FFE0001057B
:0400000300007E007B
:00000001FF
